:020000040800F2
:100000009809002045010008311B00082D1B00083D
:100010002F1B00082D1000083135000800000000DB
:10002000000000000000000000000000F91E0008B1
:100030002F10000800000000E31D00086D300008CC
:100040005F0100085F0100085F0100085F01000810
:100050005F0100085F0100085F0100085F01000800
:100060005F0100085F0100085F0100085F010008F0
:100070005F0100085F0100085F0100085F010008E0
:100080005F0100085F0100085F0100085F010008D0
:100090005F0100085F0100085F0100085F010008C0
:1000A0005F0100085F0100085F0100085F010008B0
:1000B0005F010008C13000085F0100085F0100080F
:1000C0005F0100085F0100085F0100085F01000890
:1000D0005F01000889320008F13200085933000836
:1000E000811900085F0100085F0100085F01000836
:1000F0005F0100085F0100085F0100085F01000860
:100100005F0100085F0100085F0100085F0100084F
:100110005F0100085F0100085F0100085F0100083F
:100120005F0100085F0100085F0100085F0100082F
:10013000DFF80CD000F0C4FB00480047094100087C
:10014000980900200648804706480047FEE7FEE77A
:10015000FEE7FEE7FEE7FEE7FEE7FEE7FEE7FEE777
:100160007130000831010008A0F14101192900D8BF
:100170002030704740EA01039B0703D009E008C91B
:10018000121F08C0042AFAD203E011F8013B00F85C
:10019000013B521EF9D27047D2B201E000F8012BA8
:1001A000491EFBD270470022F6E710B513460A46F7
:1001B00004461946FFF7F0FF204610BD30B505464E
:1001C0002A460B4612F8010B13F8014B08B1A04266
:1001D000F8D01CB1002802D06D1CF1E7284630BDD4
:1001E000421C10F8011B0029FBD1801A704730B562
:1001F00005460020034600E05B1C934205D2EC5C00
:10020000C85C201A01D1002CF6D130BD2DE9FE4F7B
:10021000804681EA0300C00F0C46009021F00041A7
:1002200023F00045B8EB0200A94105D24046214623
:1002300090461C460B46024623F00040104347D030
:10024000270DC7F30A00C3F30A510290401A019028
:1002500040286BDAC3F3130040F4801B00989246E9
:1002600020B10023D2EB030A63EB0B0B0198594634
:10027000C0F14002504600F0D6F906460D46504601
:100280005946019A00F0EEF910EB08006141002494
:1002900087EA115284EAE7731A4340D0009A62B3A6
:1002A000019A012A4FEA075215DC001B61EB02019B
:1002B0004FF0004202EA0752CDE90042001C41F52E
:1002C000801132462B4600F025FA03B0BDE8F08FCE
:1002D00040462146F9E7001B61EB0201001C41F595
:1002E000801300185B412018A2F5001747EB0301AB
:1002F00040EAD570B6196D4111E06D084FEA360637
:1003000045EAC0754FEA0752001B61EB0201001C71
:1003100041F5801149084FEA300000195141324639
:100320002B4603B0BDE8F04F00F0E5B9009801227C
:1003300040000023D0EB020263EBE07300982146FB
:100340004FEAE074B8EB000061EB0401E9E783F0E9
:1003500000435BE781F0004158E72DE9FE4F81EA59
:10036000030404F0004421F0004100944FF0000B1E
:1003700023F0004350EA01045ED052EA03045BD04C
:10038000C3F30A54C1F30A552C44A4F2F334019484
:10039000A0FB0254C1F3130141F48011C3F3130312
:1003A00043F4801301FB024400FB034E840A970AC6
:1003B00044EA815447EA8357A4FB076802958D0AF3
:1003C00005FB07854FEA932C04FB0C542705029D7F
:1003D0004FEA065847EA1637B5EB08056EEB070CEF
:1003E000870E920E47EA811742EA8312A7FB0201A9
:1003F000B6EB0B0164EB00042B0D43EA0C335E18E3
:1004000044EB1C50DA465146E7FB0201C5F31304E6
:100410004FEA0B3343EA14534FEA0432019C43EA98
:100420000603A4F10C040294009CCDE900B400F092
:1004300071F903B0BDE8F08F00200146F9E770B50F
:1004400021F0004303430CD0C1F30A550024D5EB3F
:10045000040564EB0403D617AD1AB34102DB002098
:10046000014670BD201841EB025170BD9623002259
:10047000114600F012B90EB5C10F80EAE0700844D1
:10048000CA07002140F233438DE80E000A460B46AE
:1004900000F040F903B000BD70B5C1F30A5201F09D
:1004A00000450024C1F3130140F2FF3341F48011F1
:1004B0009A4201DA002070BD40F233439A42A2F220
:1004C000334203DC524200F0BDF800E090402C4380
:1004D000F1D0404270BDC1F30A5210B5C1F313010F
:1004E00040F2FF3341F480119A4201DA002010BD3E
:1004F00040F233439A42A2F2334203DC524200F00C
:10050000A1F810BD904010BD00F0004230F0004056
:100510000AD0C10D01F56071C0F3160042EA015125
:10052000C208400711437047002001467047000091
:1005300030B5041E71F1000404DB4FF0004440426A
:1005400064EB0101141E73F1000405DB1C464FF03F
:100550000043524263EB0403994208BF904230BD0E
:1005600001F0004330B421F0004150EA010206D00E
:100570000A0DA2F56072C1F31301002A02DC30BC3F
:1005800000207047440F44EAC104C100E01830BCA9
:1005900000EBC25000F078B830B50B4601460020A1
:1005A0002022012409E021FA02F59D4205D303FA35
:1005B00002F5491B04FA02F52844151EA2F10102B6
:1005C000F1DC30BD2DE9F05F0546002092469B46E8
:1005D00088460646814640241BE028464146474659
:1005E000224600F02FF853465A46C01A914110D3C4
:1005F00011461846224600F016F82D1A67EB01083E
:100600004F4622460120002100F00DF817EB0009AB
:100610004E41201EA4F10104DFDC484631462A4643
:100620004346BDE8F09F202A04DB203A00FA02F19D
:10063000002070479140C2F1200320FA03F31943D0
:1006400090407047202A04DB203A21FA02F0002172
:10065000704721FA02F3D040C2F1200291400843D2
:1006600019467047202A06DBCB17203A41FA02F0E0
:1006700043EAE07306E041FA02F3D040C2F12002FF
:1006800091400843194670470029A8BF7047401C95
:10069000490008BF20F00100704710B4B0FA80FC98
:1006A00000FA0CF050EA010404BF10BC704749B1D5
:1006B000CCF1200421FA04F411FA0CF118BF012145
:1006C00021430843A3EB0C01CB1D4FEA00614FEA25
:1006D000102042BF002010BC704700EBC3501044F4
:1006E0000029A4BF10BC7047401C490008BF20F07F
:1006F000010010BC704710B5141E73F1000408DA35
:10070000401C41F1000192185B411A4301D120F0D5
:10071000010010BD2DE9F04D92469B4611B1B1FA92
:1007200081F202E0B0FA80F220329046FFF77BFFC0
:1007300004460F4640EA0A0041EA0B0153465A4676
:10074000084313D0114653EA010019D0C8F1400202
:100750005046FFF777FF05460E465046594642463B
:10076000FFF761FF084305D0012004E02046394629
:10077000BDE8F08D0020054346EAE0762C43374380
:100780000A986305E40AA0EB08000022FD0A44EA87
:1007900047540A3002D500200146E9E70105101947
:1007A0006941DDE9084500196941BDE8F04DA2E75E
:1007B0002DE9F04D81EA030404F0004B21F00045DF
:1007C00014464FF0000A23F0004150EA050220D001
:1007D00054EA01021DD0C5F30A570246C5F31303BC
:1007E000C1F31300C1F30A5640F4801543F480139B
:1007F000A7EB0608101BD64608F2FD3873EB050080
:1008000002D308F1010801E092185B41B8F1000F32
:1008100003DA00200146BDE8F08D00204FF480117E
:10082000064684460EE0171B73EB050705D3121B23
:1008300063EB050306434CEA010C49084FEA30001C
:1008400092185B4150EA0107EDD152EA030012D041
:1008500082EA040083EA0501084305D0101BAB417E
:1008600006D20122002306E000224FF0004302E0FE
:100870006FF0010253101AEB06004CEB085110EB1D
:100880000A0041EB0B01BDE8F04DFFF734BFC1F3A7
:100890000A52C1F3130140F2FF3341F480119A422E
:1008A00002DA00200146704740F233439A42A2F236
:1008B000334202DC5242FFF7C5BEFFF7B4BE000070
:1008C000064C074D06E0E06840F0010394E807009D
:1008D00098471034AC42F6D3FFF72EFC486100086D
:1008E000686100082DE9F04D00231A461B1A8A4161
:1008F00003DB00200146BDE8F08DC1F30A52C1F3CD
:10090000130141F480154FF0000BD10702D10018FC
:100910006D41521E0027044640F2FF11384601EB9C
:10092000620A3E468046024600204FF48011FFF7DF
:1009300089FEC2197141BB1846EB0100B4EB030CF0
:1009400075EB000C04D3E41A65EB000517460E4660
:10095000241908F101006D4180463428E3DDF919BE
:1009600046EB0600091BA84103D24FF0FF321346A5
:1009700001E0002213461BEB070046EB0A51BDE8DD
:10098000F04DFFF7B8BE002904D0816841F00101A5
:1009900081607047816821F001018160704700002B
:1009A00010B5154988420AD144150121204601F0AD
:1009B0003FFA2046BDE81040002101F039BA0F4946
:1009C00088420AD104150121204601F031FA20465F
:1009D000BDE81040002101F02BBA094988420AD134
:1009E0000121CC03204601F023FA2046BDE8104047
:1009F000002101F01DBA10BD002401400028014073
:100A0000003C0140014600208968490700D50120CB
:100A10007047C06C80B270470246002012680A42DC
:100A200000D001207047014600208968090700D5E1
:100A30000120704770B500240025194E01220723BC
:100A40001146304600F054F80121304600F08FF88E
:100A500002213046FFF7E0FF0028F9D03046FFF7CB
:100A6000D8FF0544022000F0E3FA641CE4B2052C30
:100A7000E4D30520B5FBF0F0FFF7F8FCFFF744FDE9
:100A80004FF06632074BFFF768FC6FF00B02FFF781
:100A9000D6FC0122FFF7D3FCBDE87040FFF760BD34
:100AA0000024014066660A4010B542680E4B1A40A9
:100AB0000C790B6842EA04221343436082680B4BB3
:100AC0001A40D1E9024323434C7942EA44021343DA
:100AD0008360C26A22F47002097C491EC9B242EAEC
:100AE0000151C16210BD0000FFFEF0FFFDF7F1FFF4
:100AF00070B5072609290AD9C568A1F10A0404EBD3
:100B00004404A640B543A3401D43C56007E0056902
:100B100001EB4104A640B543A3401D4305611F23DB
:100B2000072A09D2446B521E02EB820293409C4377
:100B300091400C43446370BD0D2A09D2046BD21F4F
:100B400002EB820293409C4391400C43046370BDCE
:100B5000C46A0D3A02EB820293409C4391400C43DD
:100B6000C46270BD816841F008018160704700294E
:100B700004D0816841F4A00181607047816821F44C
:100B8000A00181607047816841F004018160704775
:100B900030B587B001214FF4017001F03BF94FF4FB
:100BA000004001F01FF90220ADF8040000248DF888
:100BB000074001A9184800F05BFF184D2846FFF7D1
:100BC000EFFE02948DF80C408DF80D404FF460213B
:100BD0000491059401218DF8181002A92846FFF709
:100BE00063FF01212846FFF7CEFE2846FFF7BAFF34
:100BF0002846FFF718FF0028FAD12846FFF7C3FF61
:100C00002846FFF7FFFE0028FAD101212846FFF70A
:100C1000AEFF07B030BD00000008014000240140D5
:100C200010B56FF0040002F013FA09480949006892
:100C3000B0FBF1F00849C0B2087000EB4002C2EB13
:100C4000C0104FF6FF7202EAC000488010BD0000DD
:100C50000000002000127A00280000202DE9FF414A
:100C60000121182001F0D6F80121084601F0D2F840
:100C700043F20200ADF80C0010208DF80F000320A5
:100C80008DF80E00244C03A9204600F0F1FE02214D
:100C9000204600F047FF6114204600F043FFA114F6
:100CA000204600F03FFF4FF4C040ADF80C00482054
:100CB0008DF80F00194F03A9384600F0D9FE4FF404
:100CC000C06000F069FF28248DF8004000258DF8F1
:100CD00001508DF8025001268DF80360684600F03F
:100CE00029FFF003ADF80C008DF80F4003A938463A
:100CF00000F0BEFE0F21022000F0A6FE01948DF848
:100D0000085008208DF809008DF80A6001A800F04D
:100D100061FEBDE8FF810000000C014000100140B1
:100D2000012080F3138805480168054A01F4E06159
:100D300011430160BFF34F8FFEE700000CED00E0B0
:100D40000400FA057FB50121022001F055F80920C1
:100D5000ADF8080041F61F40ADF804000024ADF8DE
:100D60000A40ADF806400E4D01A9284602F03EFAB1
:100D700001224121284602F02EFA1D218DF8001093
:100D80008DF8014003218DF8021001218DF8031028
:100D9000684600F0CFFE0121284602F004FA7FBD2C
:100DA00000040040F0B587B006460121480401F078
:100DB00023F80121042001F02DF80424ADF8184097
:100DC00003258DF81A5018218DF81B101E4F06A907
:100DD000384600F04DFE0821ADF818108DF81B4084
:100DE00006A9384600F044FE4FF4A06000F0D4FE9F
:100DF00026218DF804108DF8055002208DF806008C
:100E000001208DF8070001A800F094FE0296002052
:100E1000ADF80C00ADF80E00ADF81000ADF8140000
:100E20000C20ADF81200094C02A9204602F01AFB72
:100E3000012240F22551204602F0F9FA0121204614
:100E400002F0C2FA07B0F0BD0008014000440040C3
:100E500070B586B005460121880400F0CDFF012160
:100E6000082000F0D7FF4FF48060ADF81400032491
:100E70008DF8164018218DF817101F4E05A9304621
:100E800000F0F6FDF114ADF8141004218DF81710E0
:100E900005A9304600F0ECFD4FF4A06000F07CFEA8
:100EA00027208DF800008DF801408DF802400120C8
:100EB0008DF80300684600F03DFE01950020ADF876
:100EC0000800ADF80A00ADF80C00ADF810000C20D9
:100ED000ADF80E00094C01A9204602F0C3FA012228
:100EE00040F22551204602F0A2FA0121204602F0EC
:100EF0006BFA06B070BD0000000C014000480040D5
:100F00002DE9F04105460F4600240C4E0BE0402130
:100F1000304602F065FA0028F9D0295D304602F02B
:100F200003FB641CA4B2BC42F1D34021304602F062
:100F300057FA0028F9D0BDE8F081000000480040D1
:100F400070B54FF400512C4800F0E5FD2B4C002506
:100F5000A8B1A572A089B0F5967F4BD3A07864287C
:100F600001D2401CA070FFF765FD606024498842F3
:100F70003EDD2449884205DD6420607239E00120AD
:100F8000A072E7E72049884202DD5A20607230E013
:100F90001E49884202DB502060722AE01C498842C8
:100FA00002DB4620607224E01A49884202DD3C20C0
:100FB00060721EE01849884202DD3220607218E03B
:100FC0001649884202DD2820607212E014498842E6
:100FD00002DB1E2060720CE01249884202DB142002
:100FE000607206E01049884203DB0A20607200E06C
:100FF0006572A58170BD000000100140D401002081
:10100000B81E6540B81E85405C8F82407B147E40D0
:101010009A9979408FC275405C8F7240D7A3704017
:1010200052B86E40A4706D409A996940FEE77047CF
:101030000B49498848434FF0E021486100238B6108
:10104000086940F0010008610869C20701D0C003C7
:10105000FAD5086920F0010008618B617047000033
:10106000280000200B49097848434FF0E0214861EF
:1010700000238B61086940F0010008610869C2071C
:1010800001D0C003FAD5086920F0010008618B6126
:1010900070470000280000202DE9F0412B4C01276B
:1010A000FD03207D2A4E4FF00208002816D1294664
:1010B000304600F030FD80B1C820FFF7B9FF294667
:1010C000304600F028FD48B12946304600F023FDA7
:1010D0000028F9D184F8158000E06775207D01288B
:1010E00014D12946304600F016FD78B1C820FFF72C
:1010F0009FFF2946304600F00EFD38B129463046A4
:1011000000F009FD0028F9D184F81580207D02281F
:1011100017D12946304600F0FEFC002811D0C82027
:10112000FFF786FF2946304600F0F5FC002808D07E
:101130002946304600F0EFFC0028F9D1A07A10B122
:101140006775BDE8F08103206075FAE7D4010020DF
:10115000001001402DE9F0412B4C207D627D904232
:101160004FD001273E03294D022A10D1314628468F
:1011700000F0D8FC00F01CFF227D62B13146284609
:1011800000F0D2FCA77500F0F3FD02202075607D11
:10119000012803D01EE001F099F8F3E70221284668
:1011A00000F0C0FC3146284600F0BCFC227D12B1A4
:1011B000022A03D00DE001F089F80AE0002001F0D6
:1011C00001FB01F083F8002020723146284600F030
:1011D000ABFC2775607D032813D14FF47A70FFF7BD
:1011E00027FF0221284600F09DFC3146284600F0EA
:1011F00099FC4FF40051284600F094FC0320207520
:10120000FEE7BDE8F0810000D4010020000C0140A1
:101210000FB4F0B5B3B0C82101A8FEF7C4FF002495
:1012200039AA01A8389902F099F90020009001A884
:10123000FEF7D6FF86B20D4F01AD0BE040213846D8
:1012400002F0CEF80028F9D0295D384602F06CF99A
:10125000641CA4B2B442F1D34021384602F0C0F875
:101260000028F9D033B0F0BC5DF814FB0044004016
:1012700070B590B005460E463C2101A8FEF793FFDD
:101280004FF4E130FFF78EFD4FF47A742046FFF7FC
:10129000CFFE2046FFF7CCFE09E000F0DFF9C822C0
:1012A00039A13AA000F006FB2046FFF7C1FEC82294
:1012B00035A13AA000F0FEFA0028EED1C82232A1F2
:1012C00037A000F0F7FA0028F8D1C8222EA136A0E6
:1012D00000F0F0FA0028F8D10A20FFF7A9FEC82292
:1012E00029A137A000F0E6FA0028F8D1C82226A1EB
:1012F00036A000F0DFFA0028F8D12046FFF798FE6C
:101300002046FFF795FE2046FFF792FE2046FFF7A6
:101310008FFE3C2101A8FEF746FF33462A462DA149
:1013200001A802F007F9224617A101A800F0C2FAAD
:101330000028F8D1C82214A12CA000F0BBFA002884
:10134000F8D14FF4FA7422460FA12BA000F0B2FAA4
:101350000028F8D14FF4967422460BA133A000F078
:10136000A9FA0028F8D1C82207A134A000F0A2FAF7
:101370000028F8D13449088064213448FEF713FF6F
:1013800010B0002070BD00004F4B000041542B43B3
:1013900049504D4F44453D3000000000415400008D
:1013A000415445300000000041542B554152543DFA
:1013B0003131353230302C382C312C302C3000008B
:1013C00041542B43574D4F44453D320041542B521D
:1013D0005354000041542B43575341503D22257331
:1013E000222C222573222C312C34000041542B4313
:1013F00049504D55583D300041542B4349505354AA
:101400004152543D22554450222C223235352E3241
:1014100035352E3235352E323535222C36303135B4
:10142000362C34323235342C3000000041542B43FA
:1014300049504D4F44453D310000000041542B437D
:10144000495053454E440000360000200C01002056
:1014500001460020054A1288130406D5044BC2F346
:101460000E0298541846FEF7A9BE704736000020B9
:101470000C0100202DE9F041324D288800045FD591
:10148000314C0026207802283ED1304A10787B2843
:101490003AD1A6802E4BA088115C19547D2902D028
:1014A000401CA080F7E72A4802F0AAFDE06000286F
:1014B00040D028A1274602F085FD01468069C96910
:1014C000FFF709F8B860A0F56A41FC3915D123A1EE
:1014D000F86802F077FD02691D4822A1283802F061
:1014E00029F821A1F86802F06DFD026918481DA1D4
:1014F000143802F01FF803203870F86802F03EFD3F
:1015000064211348FEF74FFE20780A2818D12A7864
:1015100062700F480D496430FEF72CFE64210B48C1
:10152000FEF741FE2E80BDE8F041094811A164306C
:10153000FEF744BE64210548FEF735FE0F480680DD
:10154000BDE8F081360000203C0000200C010020A6
:1015500028020020706F72740000000073736964C9
:10156000000000002573000070617373776F726470
:1015700000000000434C4F53454400003800002059
:1015800010B5174C2078012811D0022816D0032856
:101590001FD004280AD100F019F91249A1F1140052
:1015A00000F094F80028F8D10520207010BD0EA19D
:1015B00010A0FFF75DFE0220207010BD124C608A63
:1015C000B0F5FA6FF9D311A000F0A8F900206082FD
:1015D00010BD17A000F0A2F90420207010BD00007B
:1015E0003C00002014020020617364717765393873
:1015F000363700005869616F59695F494F545F4140
:101600006972426F78000000D40100207B22636F72
:101610006465223A2230222C226D7367223A2273AB
:101620007461727420636F6E6E656374227D000056
:101630007B22636F6465223A2231222C226D73670C
:10164000223A2267657457696669496E666F3A7314
:10165000756363657373227D0000000010B5184C3C
:101660004021204601F0BCFE0028F9D02B21204665
:1016700001F05AFF0F20FFF7DBFC4021204601F06C
:10168000AFFE0028F9D02B21204601F04DFF0F209E
:10169000FFF7CEFC4021204601F0A2FE0028F9D041
:1016A0002B21204601F040FF4FF4FA70FFF7C0FCF9
:1016B000BDE81040142203A103A000F0FBB8000015
:1016C000004400404F4B00004154000030B58FB043
:1016D00004460D463C216846FEF765FD3C21684600
:1016E000FEF761FD2B46224618A1684601F022FF55
:1016F00064221BA1684600F0DDF810B101200FB094
:1017000030BDC82219A11AA000F0D4F80028F8D1E1
:10171000C82216A119A000F0CDF80028F8D1C822DF
:1017200012A121A000F0C6F80028F8D114220FA1C0
:1017300021A000F0BFF80028F8D1224908806421D8
:101740002148FEF730FD0020D9E7000041542B432B
:10175000574A41503D222573222C22257322000036
:101760005749464920474F54204950004F4B0000ED
:1017700041542B4349504D55583D300041542B4363
:10178000495053544152543D22554450222C223149
:1017900039322E3136382E312E36222C383038362A
:1017A0002C383038362C300041542B4349504D4FA3
:1017B00044453D310000000041542B4349505345FE
:1017C0004E440000360000200C01002070B54FF49C
:1017D000E130FFF7E7FA4FF47A742046FFF728FC70
:1017E0002046FFF725FC4FF4487509E0FFF736FF68
:1017F000C8221DA11DA000F05DF82846FFF718FCC7
:10180000C82219A11DA000F055F80028EED1C82269
:1018100015A11BA000F04EF80028F8D1C82212A193
:1018200019A000F047F80028F8D10A20FFF700FCC3
:10183000C8220DA11AA000F03DF80028F8D1C82256
:1018400009A11AA000F036F80028F8D12046FFF7C9
:10185000EFFB2046FFF7ECFB2046FFF7E9FB2046B5
:10186000FFF7E6FB012070BD4F4B000041542B43B6
:1018700049504D4F44453D300000000041540000A8
:10188000415445300000000041542B554152543D15
:101890003131353230302C382C312C302C300000A6
:1018A00041542B43574D4F44453D310041542B5239
:1018B000535400002DE9F04180460F461446134D65
:1018C00000262E8064211248FEF76DFC414611A0CF
:1018D000FFF79EFCC7B18CB916E00A20FFF7A8FB02
:1018E000288800040AD53846FFF7B2FD18B12E80CB
:1018F0000020BDE8F0812E800120FAE7641E240458
:10190000240CEAD10120F4E70120F2E736000020A0
:101910000C01002025730D0A000000000FB4F0B583
:10192000B3B0C82101A8FEF73EFC002439AA01A8E3
:10193000389901F013FE0020009001A8FEF750FC3A
:1019400086B20E4F01AD0BE04021384601F048FD54
:101950000028F9D0295D384601F0E6FD641CA4B2E8
:10196000B442F1D34021384601F03AFD0028F9D0C5
:1019700033B00020F0BC5DF814FB000000440040D0
:1019800010B54FF40044204600F014F8002808D0A9
:10199000204600F009F80348007D002801D1FFF738
:1019A000BFF910BDD4010020014908607047000054
:1019B0001404014001460020054A12680A40044B05
:1019C00014331B680B4202D0002A00D0012070475C
:1019D0000004014030B51B4A83790168002B2AD0EE
:1019E00013688B431360111D0B680468A3430B60DD
:1019F000017911440B68046823430B60114C0834CF
:101A00002168036899432160231D19680568A9436B
:101A100019604179102905D011440A680068024311
:101A20000A6030BD216802681143216019680068AE
:101A30000143196030BD0079104402688A43026096
:101A400030BD00000004014010B58A07120F0F23BB
:101A5000934021F00304054921448C689C438C6029
:101A60008B68904003438B6010BD00000000014074
:101A70002DE9F0410022CC7804F00F03E40601D5F3
:101A80008C7823430C784FF00F0714F0FF0F4FF0C2
:101A9000010C1CD005680CFA02F40E882640A64200
:101AA00011D1960007FA06F825EA080503FA06F8A8
:101AB00048EA0505CE78282E02D0482E02D002E052
:101AC000446100E00461521C082AE4D305600A88DE
:101AD000FF2A1ED94568002202F108060CFA06F416
:101AE0000E882640A64210D1960007FA06F825EA8D
:101AF000080503FA06F848EA0505CE78282E00D135
:101B00004461CE78482E00D10461521C082AE3D3E8
:101B10004560BDE8F0810246002092680A4200D08C
:101B2000012070474161704701617047FEE7FEE7A1
:101B30007047000070B50F23C27801260178002A93
:101B40001ED0144A126802F4E062C2F5E062120A82
:101B5000C2F10404D3404578A54082781A402A4354
:101B6000120101F1E02181F80024007800F01F014A
:101B70008E404009800000F1E020C0F8006170BD97
:101B800001F01F0086404809800000F1E020C0F805
:101B9000806170BD0CED00E0024908430249086015
:101BA000704700000000FA050CED00E010B50021C0
:101BB000002400220378422B10D143784D2B0DD105
:101BC000435C1A4492B2491CC9B21E29F8D3C17FA2
:101BD000807F01EB0020904200D1FF24204610BD01
:101BE0002DE9F0475E4C5F4D4FF000062088000461
:101BF00019D55D48FFF7DAFFFF280FD15A48417920
:101C0000027901EB0221A984C179827901EB0221D9
:101C1000E984417A007A01EB00202885268064213E
:101C20005148FEF7C0FA288AB0F5FA6F03D3E220D4
:101C300000F0AEF82E82E98BA88C6427DFF82C81A7
:101C40000A266FF0130A4FF48279814228D0B8F83F
:101C500000100AEB9104B0FBF7F0C2B204F10800E7
:101C600080B21032494600F00FFFA88CB0FBF6F0AE
:101C7000B0FBF6F106FB110204F1100080B2103245
:101C8000494600F001FFA88CB0FBF6F106FB1102FB
:101C90001834A0B21032494600F0F6FEA88CE88352
:101CA000298CE88C81422AD0B8F800100AEB510444
:101CB0004FF0500AB0FBF7F0C2B204F1080080B256
:101CC0001032514600F0E0FEE88CB0FBF6F0B0FBBD
:101CD000F6F106FB110204F1100080B210325146F9
:101CE00000F0D2FEE88CB0FBF6F106FB11021834CE
:101CF000A0B21032514600F0C7FEE88C2884288D2F
:101D0000698C88422AD0B8F80010890801EB410498
:101D1000103CB0FBF7F0C2B204F1080080B2103200
:101D2000494600F0B1FE288DB0FBF6F0B0FBF6F1AD
:101D300006FB110204F1100080B21032494600F097
:101D4000A3FE288DB0FBF6F106FB11021834A0B2F9
:101D50001032494600F098FE288D6884BDE8F0876F
:101D600038000020D4010020700100208C030020E6
:101D700010B54FF41650FFF76BF802210348FFF738
:101D8000D3FEBDE810401420FFF752B9000C01400B
:101D900030B585B00546002414216846FEF703FAE5
:101DA000002142228DF800204D228DF801208DF86F
:101DB000025000208DF803008DF804006846425C54
:101DC000224494B2491CC9B20529F8D3200A8DF8DF
:101DD00005008DF8064007216846FFF791F805B029
:101DE00030BD7047034A516821F4404101435160BE
:101DF0007047000000100240054A002903D0D16955
:101E00000143D1617047D1698143D16170470000BE
:101E100000100240054A002903D0916901439161F5
:101E20007047916981439161704700000010024042
:101E3000054A002903D0D1680143D1607047D168B9
:101E40008143D160704700000010024010B5264A5F
:101E5000516801F00C01254B002927D0042927D017
:101E6000082927D00360516801F0F0010909204BCF
:101E70005C5C0168E1404160546804F4E064240A59
:101E80001C5D21FA04F48460546804F46054E40A8C
:101E90001B5DD940C160526802F44042920B144B62
:101EA0001B1F9A5CB1FBF2F1016110BD0360DAE720
:101EB0000360D8E7516801F47011536803F480336C
:101EC000022404EB914133B153689B0307D5094BBE
:101ED00059430160C7E7074B59430160C3E7034B10
:101EE00059430160BFE700000010024000127A0071
:101EF0001800002000093D00704700F001B8000004
:101F00000CB50022019200922748016841F480310B
:101F100001604FF4A063016801F400310091019960
:101F2000491C0191009911B901999942F3D10168B5
:101F3000890302D50121009100E000920099012956
:101F400030D11A490A6842F010020A600A6822F089
:101F500003020A600A6842F002020A6041684160B6
:101F600041684160416841F480614160416821F409
:101F70007C114160416841F4E8114160016841F021
:101F80008071016001688901FCD5416821F003017D
:101F90004160416841F0020141604168C1F3810143
:101FA0000229FAD10CBD00000010024000200240BE
:101FB0002DE9F0412D4C2088400861880325B1FBB4
:101FC000F5F10A3189B22A4E47F6FF7232805A2360
:101FD000642200F0B1FC2088800800EB400061889A
:101FE0000627B1FBF7F2B1FBF5F102EB410189B233
:101FF0004FF6E07232802D23322200F09DFC2088C3
:1020000080086188B1FBF7F2B1FBF5F102EB410109
:1020100089B248F21F4232802D23322200F08CFC1C
:1020200020886FF0170101EB500080B2282100F0EA
:1020300004FF20886FF0130505EB500080B2B42137
:1020400000F020FF208805EB900080B2E6252946AD
:1020500000F0CEFE2088800800EB4000103880B2EF
:102060002946BDE8F04100F0A5BE00008C03002029
:102070004E0000202DE9F041914FF889B0F5FA7F2C
:102080007BD3B878022878D300243846B97A007D0B
:10209000012903D110B14FF4FC6403E0022801D1FF
:1020A0004FF6FF74787A397A002688427ED0DFF8BE
:1020B000148250282ED3A8F800400C242346CD22A9
:1020C0002146CA2000F0DEFB641CE4B2132CF5D3D9
:1020D0000C242346D2222146CF2000F0D3FB641CDF
:1020E000E4B2132CF5D30C242346D7222146D42066
:1020F00000F0C8FB641CE4B2132CF5D30C24234677
:10210000DC222146D92000F0BDFB641CE4B2132C74
:10211000F5D3CAE03C2831D3A8F800600C252B4643
:10212000CD222946CA2000F0ADFB6D1CEDB2132D67
:10213000F5D3A8F800400C242346D2222146CF2014
:1021400000F0A0FB641CE4B2132CF5D30C2423464E
:10215000D7222146D42000F095FB641CE4B2132C56
:10216000F5D30C242346DC222146D92000F08AFB3B
:10217000641CE4B2132CF5D397E09EE0282832D3F8
:10218000A8F800600C252B46CD222946CA2000F075
:1021900079FB6D1CEDB2132DF5D30C252B46D22205
:1021A0002946CF2000F06EFB6D1C00E084E0EDB20C
:1021B000132DF3D3A8F800400C242346D722214640
:1021C000D42000F05FFB641CE4B2132CF5D30C2484
:1021D0002346DC222146D92000F054FB641CE4B2E3
:1021E000132CF5D361E0142830D3A8F800600C2537
:1021F0002B46CD222946CA2000F044FB6D1CEDB2CF
:10220000132DF5D30C252B46D2222946CF2000F0E2
:1022100039FB6D1CEDB2132DF5D30C252B46D722BF
:102220002946D42000F02EFB6D1CEDB2132DF5D302
:10223000A8F800400C242346DC222146D92000F0D7
:1022400021FB641CE4B2132CF5D32EE068B3A8F88C
:1022500000600C242346CD222146CA2000F012FB48
:10226000641CE4B2132CF5D30C242346D22221465D
:10227000CF2000F007FB641CE4B2132CF5D30C2430
:102280002346D7222146D42000F0FCFA641CE4B295
:10229000132CF5D30C242346DC222146D92000F050
:1022A000F1FA641CE4B2132CF5D34FF480510648C4
:1022B000FFF73AFC787A3872FE81BDE8F0810000C1
:1022C000D40100204E000020000C014010B5184938
:1022D0004FF6FF7008800923DE221946C82000F05F
:1022E000D1FA1523DE221946C82000F0CBFAC82205
:1022F00015230921104600F0C5FADE221523092115
:10230000104600F0BFFA0D23C8221946C52000F080
:10231000B9FAC52211230D21104600F0B3FA11239A
:10232000C822BDE810401946C52000F0ABBA000035
:102330004E00002070B5404D288BB0F5FA6F7AD36F
:102340000024A87D3D49002647F6FF72012808D0E9
:10235000022814D0032821D004282ED005283BD0F1
:1023600068E00A80234620222146002000F08AFAF5
:10237000641CE4B20D2CF5D30220A8755AE00A8043
:102380000F24234618222146002000F07BFA641C0B
:10239000E4B21C2CF5D30320A8754BE00A801E2460
:1023A000234610222146002000F06CFA641CE4B29F
:1023B0002B2CF5D30420A8753CE00A802D2423465D
:1023C00008222146002000F05DFA641CE4B23A2C99
:1023D000F5D30520A8752DE00E8023462022214646
:1023E000002000F04FFA641CE4B20D2CF5D30F244A
:1023F000234618222146002000F044FA641CE4B26F
:102400001C2CF5D31E24234610222146002000F068
:1024100039FA641CE4B22B2CF5D32D242346082270
:102420002146002000F02EFA641CE4B23A2CF5D3C9
:102430000120A8752E8370BDD40100204E0000201D
:1024400010B5112000F044FD1420FEF7F1FDD0205E
:1024500000F03EFD072000F05DFD422000F05AFD37
:102460001D2000F057FDD12000F032FD002000F0CB
:1024700051FD1A2000F04EFD092000F04BFDD22046
:1024800000F026FD012000F045FD222000F042FD75
:10249000C02000F01DFD102000F03CFD3B2000F0AE
:1024A00039FD002000F036FD022000F033FD112040
:1024B00000F030FDC52000F00BFD032000F02AFDE8
:1024C000C82000F005FD002000F024FD252000F0CC
:1024D00021FD212000F01EFD052000F01BFD002045
:1024E00000F018FD0A2000F015FD652000F012FD37
:1024F000252000F00FFD772000F00CFD502000F0AB
:1025000009FD0F2000F006FD002000F003FDF8207B
:1025100000F0DEFC012000F0FDFCFE2000F0D8FC05
:10252000002000F0F7FC022000F0F4FC202000F076
:10253000CFFC362000F0CCFC082000F0EBFC3A2069
:1025400000F0C6FC552000F0E5FC2B2000F0C0FC9C
:10255000002000F0DFFC002000F0DCFC012000F097
:10256000D9FC3F2000F0D6FC2A2000F0B1FC00206E
:1025700000F0D0FC002000F0CDFC012000F0CAFCEF
:10258000DF2000F0C7FC7820FEF752FDBDE81040C8
:10259000292000F09DBC10B5CF2000F099FC002050
:1025A00000F0B8FCC12000F0B5FC302000F0B2FC17
:1025B000ED2000F08DFC642000F0ACFC032000F066
:1025C000A9FC122000F0A6FC812000F0A3FCE8206A
:1025D00000F07EFC852000F09DFC102000F09AFCAD
:1025E0007A2000F097FCCB2000F072FC392000F03C
:1025F00091FC2C2000F08EFC002000F08BFC34209D
:1026000000F088FC022000F085FCF72000F060FC60
:10261000202000F07FFCEA2000F05AFC002000F0AF
:1026200079FC002000F076FCC02000F051FC1B205B
:1026300000F070FCC12000F04BFC012000F06AFCAF
:10264000C52000F045FC302000F064FC302000F094
:1026500061FCC72000F03CFCB72000F05BFC36209A
:1026600000F036FC482000F055FC3A2000F030FC29
:10267000552000F04FFCB12000F02AFC002000F0B3
:1026800049FC1A2000F046FCB62000F021FC0A208C
:1026900000F040FCA22000F03DFCF22000F018FC0D
:1026A000002000F037FC262000F012FC012000F092
:1026B00031FCE02000F00CFC0F2000F02BFC2A2065
:1026C00000F028FC282000F025FC082000F022FC67
:1026D0000E2000F01FFC082000F01CFC542000F02D
:1026E00019FCA92000F016FC432000F013FC0A207E
:1026F00000F010FC0F2000F00DFC002000F00AFCA0
:10270000002000F007FC002000F004FC002000F096
:1027100001FCE12000F0DCFB002000F0FBFB1520B9
:1027200000F0F8FB172000F0F5FB072000F0F2FBAB
:10273000112000F0EFFB062000F0ECFB2B2000F056
:10274000E9FB562000F0E6FB3C2000F0E3FB05200F
:1027500000F0E0FB102000F0DDFB0F2000F0DAFBC2
:102760003F2000F0D7FB3F2000F0D4FB0F2000F00B
:10277000D1FB2B2000F0ACFB002000F0CBFB0020B5
:1027800000F0C8FB012000F0C5FB3F2000F0C2FBB9
:102790002A2000F09DFB002000F0BCFB002000F090
:1027A000B9FB002000F0B6FBEF2000F0B3FB1120D6
:1027B00000F08EFB7820FEF73BFCBDE8104029209E
:1027C00000F086BB70B5064600240948018845889C
:1027D0004D430021084600F077FA00F0BDFB03E00E
:1027E000304600F097FB641CAC42F9D370BD00008A
:1027F0008C0300202DE9F003214A2C272A252B26C3
:1028000091884FF0F00C49F241384FF4A07446F62D
:10281000040300280CD0994227D001209071148025
:10282000A2F802C0414516D1D771157256721CE04C
:1028300000209071A2F800C05480414501D0994217
:1028400013D1D7711572567299420ED114804FF47C
:10285000F070508009E02220A1F50943893B09D09E
:10286000D0712120107220205072BDE8F0030020AA
:1028700000F07CB9D0714F2010724E205072F4E7F6
:102880008C0300202DE9FE4F4FF0000B00250026A1
:10289000171AA3EB010881468A46681E002F03DD44
:1028A0004FF00101019107E003D14FF000010191C8
:1028B00002E00190C7F10007B8F1000F03DD4FF00F
:1028C0000100009007E003D14FF00000009002E00B
:1028D0000090C8F10008474501DD3C4600E0444651
:1028E000601C029015E01FFA8AF11FFA89F000F0CF
:1028F00015F83D444644A54202DD2D1B0198814454
:10290000A64202DD361B009882440BF1010B1FFA30
:102910008BFB02988345E6DDBDE8FE8F10B500F025
:10292000D3F900F019FB03484088BDE8104000F0DF
:10293000F1BA00004C0000202DE9FC5F80468B4678
:1029400017469A4229D302FB02FA5B430093ABEB92
:10295000070085B20BEB070001901BE0A8EB070016
:1029600084B208EB0709A5EB0B060FE0A4EB080007
:10297000404306FB0600504506D80099884203D91B
:1029800029462046FFF7CAFF641CA4B2A145EDD832
:102990006D1CADB20198A842E0D8BDE8FC9F0000D4
:1029A000F8B501211C20FFF735FA4FF47070ADF82F
:1029B000000010208DF8030003208DF80200694606
:1029C0002F48FFF755F82E484FF400711030016082
:1029D00040210160802101608115016000F0FAFA58
:1029E0003220FEF725FB3220FEF722FB254C46F66F
:1029F000040649F24135A088FF2806D3A0F57F419F
:102A0000FF3902D0B0F5134F29D1D32000F060FA7E
:102A100000F08CF800F08AF800F088F80002A0803E
:102A200000F084F8A188C0B20843A080A84210D06A
:102A3000BF2000F04DFA00F079F800F077F800F0D0
:102A400075F80002A08000F071F8A188C0B20843B8
:102A5000A080A088A84202D0B04200D0A580A08863
:102A6000A84202D1FFF797FD03E0B04201D1FFF782
:102A7000E7FC0020FFF7BEFE0020FFF7A3FEF8BD35
:102A8000000C01408C0300202DE9F84F07460C464E
:102A90004FF00008A1462248DFF888A000EB0210A2
:102AA000DFF884B00090009810F808600025300628
:102AB00004D54FF6FF70AAF8020002E00020AAF841
:102AC000020021463846FFF729FF7006060E641CF7
:102AD000A4B2BBF80000B84205D84FF6FF70AAF8C0
:102AE0000200BDE8F88FA4EB090010280BD06D1C84
:102AF000EDB2082DDBD308F1010808F0FF08B8F1AA
:102B0000100FD0D3EDE74C467F1CBFB2BBF80000DE
:102B1000B842F0D84FF6FF70AAF80200E1E70000D3
:102B2000885600084C0000208C0300202DE9F0415D
:102B300000F028FA0C4C4FF4807020608020206058
:102B40004026201D0660451505600120FEF78AFA23
:102B500000F008FA07460120FEF784FA2660256097
:102B60003846BDE8F0810000100C014070B500242B
:102B7000544D46F604022946AB798988012B18D1B9
:102B8000914216D0082814D2DFE800F00406080AA3
:102B90000C0E101206200CE007200AE0042008E0CA
:102BA000052006E0012004E0002002E0032000E010
:102BB0000220A1F51343413B01D0914259D108288D
:102BC00012D2DFE800F0110406080A0C0E1080246F
:102BD0000AE0402408E0C02406E0202404E0602449
:102BE00002E0A02400E0E024362044F008049142F2
:102BF00001D144F0020400F06BF9204600F08AF99C
:102C0000A00606D528886988884208D2298068806D
:102C100005E028886988884201D929806880287A57
:102C200000F056F9002000F075F9002000F072F96C
:102C30002888401EC0F30F2000F06CF92878401E51
:102C4000C0B200F067F9687A00F042F9002000F0A5
:102C500061F9002000F05EF96888401EC0F30F2083
:102C600000F058F9A878BDE87040401EC0B200F0EE
:102C700051B9082812D2DFE800F0040608110A0C46
:102C80000E1030240AE0102408E0202406E0382446
:102C900004E0282402E0182400E00824A1F50940FB
:102CA000893809D0032044F4805400F011F92046FB
:102CB000BDE8704000F02EB9112046F240010C43EF
:102CC000F3E700008C03002070B504460E461A4D51
:102CD0002846AA88007AA2F51341413907D0A2F507
:102CE000D041043903D0A979012913D016E000F0AE
:102CF000EFF8200A00F00EF9E0B200F00BF9687A64
:102D000000F0E6F8300A00F005F9F0B2BDE87040D6
:102D100000F000B92988091B491E8CB200F0D8F8D0
:102D2000204600F0F7F8287A00F0D2F83046BDE8E7
:102D3000704000F0EFB800008C0300202DE9F84F40
:102D400082460C460027A046184902EBC20001EB60
:102D50008000DFF85C9000900098C65D00254FF67B
:102D6000FF7B300602D5A9F802B002E00020A9F8E6
:102D7000020021465046FFF7D1FD7006060E641C86
:102D8000A4B2A4EB0800182809D06D1CEDB2082DE0
:102D9000E7D37F1CFFB2242FDED3BDE8F88F444673
:102DA0000AF1010A1FFA8AFAF3E70000785C0008CA
:102DB0004C00002070B504460D46302229462046BE
:102DC000FFF762FE04F1080080B22D222946FFF7CA
:102DD0005BFE04F1100080B211222946FFF754FE79
:102DE0001834A0B22946BDE870401022FFF74CBE4F
:102DF00070B504460D46302229462046FFF744FEB2
:102E000004F1080080B22D222946FFF73DFE04F1AF
:102E1000100080B211222946FFF736FE04F1180097
:102E200080B20E222946FFF72FFE2034A0B2294699
:102E3000BDE870401022FFF727BE70B504460D466E
:102E4000002229462046FFF779FF04F10C0080B2EA
:102E500001222946FFF772FF04F1180080B2022216
:102E60002946FFF76BFF04F1240080B203222946B4
:102E7000FFF764FF3034A0B22946BDE87040042259
:102E8000FFF75CBF70B504460D4655222946204623
:102E9000FFF7FAFD04F1080080B247222946FFF748
:102EA000F3FD04F1100080B20F222946FFF7ECFD7C
:102EB00004F1180080B24D222946FFF7E5FD2034C9
:102EC000A0B22946BDE870401322FFF7DDBD000027
:102ED0002DE9F041064600F07DF80D4C4FF480706E
:102EE00020604020251F2860C70027600120FEF7D2
:102EF000B9F8304600F096F80120FEF7B3F88026C6
:102F000026600120FEF7AEF82E602F60BDE8F0814C
:102F1000140C01402DE9F041064600F05BF80D4C21
:102F20004FF48070206040202060C500271D3D6068
:102F30000120FEF797F8304600F074F80120FEF704
:102F400091F880263E600120FEF78CF8266025600F
:102F5000BDE8F081100C01400148C079FFF7B8BF0F
:102F60008C03002005488068C1B2054800684FF412
:102F70007F4202EAC000084480B27047001001405E
:102F800008080140F8B5104C207801281AD0FF201D
:102F9000ADF8000004268DF8036003258DF802507B
:102FA00069460A48FEF764FD4FF4FF50ADF8000093
:102FB0008DF803608DF8025069460548FEF758FD0C
:102FC00001202070F8BD00004C00002000100140DE
:102FD00000080140F8B5104C207802281AD0FF20D4
:102FE000ADF8000010268DF8036003258DF802501F
:102FF00069460A48FEF73CFD4FF4FF50ADF800006B
:103000008DF803608DF8025069460548FEF730FDE3
:1030100002202070F8BD00004C000020001001408C
:1030200000080140C1B2084A1161C943C9B25161E7
:10303000010A4901054A11606FEA10200006C00C20
:10304000111D086070470000001001401008014089
:103050004FF0E021042804D0086920F00400086142
:103060007047086940F0040008617047704700002D
:1030700010B50F48016841F00101016041680D4A37
:103080001140416001680C4A11400160016821F45F
:1030900080210160416821F4FE0141604FF41F016D
:1030A0008160FEF72AFF05494FF00060086010BDFF
:1030B000001002400000FFF8FFFFF6FE08ED00E000
:1030C00010B5324C0121204600F079F800285CD080
:1030D0000121204600F064F82D4C2E4B0021208861
:1030E000A8B1020413D41A78C82A01D8521C1A7045
:1030F0001A78142A0DD35A88824205D140F4004030
:1031000020805980197004E05880197001E019700E
:103110005980214C2088A8B1020413D45A78642A1B
:1031200001D8521C5A705A78142A0DD39A888242B8
:1031300005D140F4004020809980597004E09880C7
:10314000597001E05970998014494FF6E852088A85
:10315000904201D2401C0882C889904201D2401C92
:10316000C8818889904201D2401C8881088B904296
:1031700001D2401C0883888B904201D2401C888376
:10318000488A904201D2401C488210BD0004004091
:10319000360000202C00002038000020D401002040
:1031A000C94301827047002904D0018841F0010120
:1031B00001807047018821F00101018070470246BB
:1031C0000020138A0B4092890A40002B02D0002A6B
:1031D00000D001207047002A03D082890A438281EF
:1031E000704782898A4382817047000030B5028827
:1031F0001B4C1C4DA0420DD0A8420BD0B0F1804F0B
:1032000008D0194B984205D0184B984202D0184B61
:10321000984203D122F070034A881A43154B984212
:1032200006D0154B984203D022F44073CA881A4343
:1032300002808A8882850A880285A0420AD0A84234
:1032400008D00E4A904205D00D4A904202D00D4A55
:10325000904201D1097A01860121818230BD0000AE
:10326000002C0140003401400004004000080040F0
:10327000000C0040001000400014004000400140DD
:10328000004401400048014070B5164C40F22555FD
:103290002946204600F0ABF888B1204600F040F9FE
:1032A000C3B211480288110409D410498B54521C2E
:1032B00092B202805A2A02D342F4004101800821CE
:1032C000204600F08DF8012806D1204600F028F9AC
:1032D0000821204600F074F829462046BDE87040D9
:1032E00000F06EB800380140320000206C00002071
:1032F00070B5164D40F225563146284600F077F855
:1033000088B1284600F00CF9C4B211490B881804A2
:1033100009D4581C82B20F480A80C4545A2A02D3D6
:1033200042F4004008800821284600F059F801289E
:1033300006D1284600F0F4F80821284600F040F8AD
:1033400031462846BDE8704000F03AB800440040DD
:10335000360000200C01002070B5164C40F22555B7
:103360002946204600F043F888B1204600F0D8F8FE
:10337000C3B211480288110409D410498B54521C5D
:1033800092B202803B2A02D342F40041018008211C
:10339000204600F025F8012806D1204600F0C0F8AC
:1033A0000821204600F00CF829462046BDE8704070
:1033B00000F006B80048004034000020D000002093
:1033C0008A05C94301807047002904D0818941F4EE
:1033D000005181817047818921F4005181817047BA
:1033E0000246002012880A4200D00120704770B5C2
:1033F000002440F66A12C1F3421301F01F050126B2
:1034000006FA05F2012B0CD0022B0DD0838A134053
:10341000090A8E40008830400BB100B101242046DB
:1034200070BD83891340F3E7038A1340F0E710B5BA
:1034300040F66A13C1F3421301F01F040121A140B9
:10344000012B07D0022B07D014303AB102680A438F
:10345000026010BD0C30F8E71030F6E702688A43CE
:10346000026010BD30B585B004460D46208A4CF68A
:10347000FF710840E98801432182A0894EF6F311CB
:103480000840A9882A8911436A8902431143A1810E
:10349000A08A4FF6FF410840A9890143A1826846EE
:1034A000FEF7D4FC1D48844201D1039800E0029845
:1034B000A189090408D500EBC00101EB00102968BF
:1034C0004900B0FBF1F007E000EBC00101EB001098
:1034D00029688900B0FBF1F06422B0FBF2F1090128
:1034E0000B096FF018056B4300EB8300A3891D04E3
:1034F0004FF0320307D503EBC000B0FBF2F000F051
:103500000700084306E003EB0010B0FBF2F000F008
:103510000F000843208105B030BD00000038014095
:103520008088C0F308007047C1F3080181807047AC
:10353000FEE700000FB4084B10B504A902AA0398D7
:1035400000F080F9044602A9002000F012FD204698
:1035500010BC5DF814FB0000733F000837B514463B
:103560000846064B6A46214600F06CF90446694657
:10357000002000F0FEFC20463EBD0000733F000826
:10358000490050EAC12018BF04204A0D18BF40F07E
:10359000010040F2FF72B2EB515F08BF40F0020041
:1035A000012808BF052070472DE9F0414F1E00EBB0
:1035B000C7010446D1E9000115461E4637F0060250
:1035C0000DD02A463346FCF7C8FE7F1E04EBC70326
:1035D000D3E90023FCF71AFE37F00602F1D1022FDF
:1035E00025D0042F13D0062F18BFBDE8F0812A463E
:1035F0003346FCF7B2FED4E90A23FCF707FE2A465D
:103600003346FCF7AAFED4E90823FCF7FFFD2A465F
:103610003346FCF7A2FED4E90623FCF7F7FD2A4661
:103620003346FCF79AFED4E90423FCF7EFFD2A4663
:103630003346FCF792FED4E90223FCF7E7FD2A4665
:103640003346FCF78AFED4E90023BDE8F041FCF7DD
:10365000DDBD00000022134610460149FDF7A8B861
:103660000000F03FFCF7D2BD002213461046114681
:10367000FDF79EB840F2013200204FF0E041FCF728
:10368000DEBE0000024A00201107FCF7D8BE000091
:1036900001FDFFFF02E008C8121F08C1002AFAD18D
:1036A00070477047002001E001C1121F002AFBD1C2
:1036B0007047000001490860704700006800002062
:1036C0002DE9FF5F82B00021DDE90430020DDDF855
:1036D00040B0034318D044F61050A2F2FF324243E8
:1036E0001514119801281FD0A5EB0B00401C5FEAB0
:1036F000000A4FF000064E4FDFF83891B0465046B2
:1037000015D5CAF1000413E0119801244AA3012839
:1037100001D16FEA0B010298119AC0E90031C0E9AA
:10372000024206B0BDE8F09FCBF10000DFE704469F
:103730000021404A491842EB0450CDE9001012E044
:10374000E00707D032463B4640464946FCF705FEB7
:103750008046894632463B4610461946FCF7FDFD39
:1037600006460F466410002CEAD1DDE90401DDE9CC
:103770000023BAF1000F06DAFCF7EFFD42464B4694
:10378000FCF7EBFD05E0FDF713F842464B46FDF76D
:103790000FF804460E460022284BFCF7C9FE03D85A
:1037A0004FF0FF30014607E00022254B204631460E
:1037B000FCF72CFDFDF76BF8102409E0002C0ADB68
:1037C0000A220023FCF7FEFE039B30321A55641ECA
:1037D00050EA0102F2D1641C039AC4F111031444AB
:1037E000119A012A03D0012208430DD10AE00843AF
:1037F00004D000204FF0110B119072E7A3EB0B05E2
:103800006D1E0DE05B4504DD4FF0000205F1010582
:1038100004E003DA4FF00002A5F10105002AECD024
:1038200002981199C0E90231C0E9004579E700002A
:10383000000014400000F03F300000000000F043A2
:103840000000E03F2DE9FF4F95B09B4689460646B4
:1038500000250FE2252877D100242746F84A0121C8
:10386000059400E0044316F8013F203B01FA03F001
:103870001042F7D130782A2811D06FF02F0330781A
:10388000A0F13002092A16D8059A44F0020402EB8E
:10389000820203EB42021044761C0590EFE759F8D0
:1038A000042B0592002A03DA504244F40054059098
:1038B00044F00204761C30782E2816D116F8010F39
:1038C00044F004042A280DD06FF02F023078A0F1C4
:1038D0003003092B09D807EB870302EB4303C71812
:1038E000761CF3E759F8047B761C30786C280FD0EF
:1038F00006DC4C2817D068280DD06A2814D104E0C3
:10390000742810D07A280FD10DE044F400140AE096
:1039100044F4801401E044F440147278824202D1ED
:1039200004F58014761C761C307866280BD013DCE6
:10393000582877D009DC002875D04528F6D04628CD
:10394000F4D047281AD19DE118E0632835D06428C7
:1039500079D0652812D195E1702873D008DC6728EA
:10396000F1D069286FD06E280DD06F2806D1B5E050
:1039700073282CD0752875D0782874D05A4617999A
:1039800090476D1C75E1C4F30250022809D003284A
:103990000DD0D9F8001004280DD00D6009F10409EC
:1039A00067E1D9F80010EA17C1E90052F6E7D9F843
:1039B00000100D80F2E70D70F0E719F8041B8DF888
:1039C000001000208DF80100EA46012003E059F8BC
:1039D00004AB4FF0FF3061074FF0000102D40DE05F
:1039E00008F101018846B9420FDA8045F8DB1AF880
:1039F00008100029F4D108E008F10101884681424D
:103A0000FADB1AF808100029F6D105985B46A0EBFE
:103A1000080721463846179A00F094FA284400EB2C
:103A2000080507E04DE029E10DE01AF8010B5A46C0
:103A300017999047B8F10108F7D25B4621463846FE
:103A4000179A13E142E00A220092C4F302524FF0A7
:103A5000000A022A08D059F804CB032A4FEAEC7175
:103A60000AD00DE029E02AE009F1070121F0070260
:103A7000F2E802C1914609E00FFA8CFC4FEAEC71C2
:103A8000042A03D14FFA8CFC4FEAEC71002907DAC3
:103A90000A460021DCF1000C61EB02012D2202E05C
:103AA000220504D52B228DF80420012203E0E20731
:103AB00001D02022F7E7904659E00A2102E01022C7
:103AC0000DE010214FF0000A00910BE010224FF0A2
:103AD000000A44F004040827009203E008224FF093
:103AE000000A0092C4F30252022A05D059F804CB0E
:103AF0000021032A08D009E009F1070121F007029B
:103B0000F2E802C1914605E01FFA8CFC042A01D1BB
:103B10000CF0FF0C4FF00008220728D5702806D0C3
:103B2000009B83F0100353EA0A0305D00EE0402205
:103B30008DF80420012208E05CEA010206D0302260
:103B40008DF804208DF8050002229046009B83F03A
:103B5000080353EA0A030AD15CEA010201D16207B1
:103B600005D530228DF804204FF001087F1E58281B
:103B700004D034A003900EA802900DE036A0F9E71F
:103B800053466046009AFCF71DFD84460398825C0C
:103B90000298401E029002705CEA0100F0D1029887
:103BA00006A9081A00F1200A600702D524F480341F
:103BB00000E00127574502DDA7EB0A0000E00020E6
:103BC00000EB0A01009005984144401A0590E0037B
:103BD00006D45B462146179A059800F0B3F90544D0
:103BE000002706E001A85A46C05D179990476D1C52
:103BF0007F1C4745F6DBE0030CD55B462146179A50
:103C0000059800F09FF9054404E030205A461799C2
:103C100090476D1C0099481E00900029F5DC08E0D3
:103C2000029802995A460078491C029117999047C8
:103C30006D1CBAF10001AAF1010AF1DC65E1000096
:103C40000928010030313233343536373839616272
:103C50006364656600000000303132333435363736
:103C600038394142434445460000000000F058F90D
:103C70000544761C307800287FF4ECAD19B0284656
:103C8000BDE8F08F620700D4062709F1070222F091
:103C9000070CFCE80223E14603F000485FEA080C49
:103CA00002D00FF2702C0DE05FEA045C02D50FF237
:103CB000682C07E05FEAC47C02D00FF2602C01E0C0
:103CC000AFF2700C4FF0FF3823F00043CDF850C036
:103CD00065280CD006DC452809D046281DD0472889
:103CE0003DD13DE0662818D067287ED138E000211C
:103CF000112F01DB112000E0781CCDE9000106A99D
:103D00000EA8FFF7DDFCDDE90F010E9A03910021FB
:103D1000009207F1010A04914DE04FF00040009736
:103D2000CDE9011006A90EA8FFF7CAFCDDE90F02D4
:103D300003920E9B11990022DDF80CA000930492CF
:103D400011B9791C00EB010AB7EB0A0004D4C0F1E9
:103D5000FF3007F1010A0490AAEB0700019044E04C
:103D6000012F00DA01270021112F01DD112000E0D1
:103D70003846CDE9000106A90EA8FFF7A1FCDDE950
:103D80000F010E9A0391002104910092BA46210777
:103D90000CD40399514500DA8A46BAF1010F05DDCA
:103DA000009AAAF10101515C302908D0B84202DA28
:103DB00010F1040F06DA0121CDE9011015E0AAF196
:103DC0000101E9E7002805DC049901440491AAEB0C
:103DD000000102E0411C514500DD8A460499401A69
:103DE000401C01904FF000400290200704D401983D
:103DF000504501DBCDF8048000208DF84F0002987B
:103E00000DF14F07B0F1004F25D02B200E900298F6
:103E10004FF0020800280CDA404202902D200E904C
:103E200007E00A210298FCF7B7FB3031029007F84F
:103E3000011DB8F10001A8F10108F2DC0298002888
:103E4000EFD1791E0E980870307800F0200040F015
:103E5000450007F8020D12A8C01B00F107081498CE
:103E6000007800B1012000EB0A01019801EBE0713C
:103E700005984144401A401E0590E00306D45B4675
:103E80002146179A059800F05DF8054414980078CB
:103E900018B15A46179990476D1CE00324D55B462C
:103EA0002146179A059800F04DF805441CE0049847
:103EB000002807DBDDE90301884203DD0098405C50
:103EC000179901E0179930205A469047049805F158
:103ED0000105401C04900198401E019004D12E2041
:103EE0005A46179990476D1CBAF10001AAF1010AD0
:103EF000DDDC05E017F8010B5A46179990476D1C59
:103F0000B8F10001A8F10108F4DC5B462146179ADC
:103F10000598ABE62D0000002B00000020000000FB
:103F20002DE9F041044600251E461746880404D4B6
:103F300005E039462020B0476D1C641EF9D528469F
:103F4000BDE8F0812DE9F041044600251E4690466B
:103F5000C80301D5302700E02027880404D505E0F8
:103F600041463846B0476D1C641EF9D52846BDE869
:103F7000F0810A68531C0B601070704770B50446DE
:103F80000F4E19E02568A089C00503D4A06808B1C8
:103F9000FFF7F4FFA089C00503D4206908B1716858
:103FA0008847A089800503D4206A08B171688847D2
:103FB0007168204688472C46002CE3D170BD000074
:103FC0005400002070B50D46846800E024682CB1D0
:103FD0002946206A00F04AF80028F7D1204670BD33
:103FE00010B5064928200968884704461CB12821D5
:103FF0002046FCF7D8F8204610BD000054000020F1
:1040000000221146AFF300802DE9F04104460D4631
:104010009046FFF7E5FF0646134F0020B860C6B193
:10402000204601F0C7F80146304600F079FB04460F
:104030008CB1B8F1000F13D0204601F0BBF8044654
:10404000207868B13046FFF799FFBC600020BDE8DA
:10405000F0810020FBE73046FFF790FF0020F6E7F5
:1040600005B12C603046F2E75400002070B50446DC
:104070000D46002C01D02DB10AE00DB1012070BD1C
:10408000002070BD012070BD207898B1641C6D1CAB
:104090002078FCF769F806462878FCF765F8864230
:1040A000F2D02078FCF760F804462878FCF75CF83A
:1040B000201A70BD002070BD10B5002821D0114B12
:1040C0000022001F196803E0814203D80A464968AC
:1040D0000029F9D152B11368841A9C4204D10068B6
:1040E00018441060104602E0506000E0186039B1DA
:1040F00002680B1A934203D10B681A4402604968A4
:10410000416010BD60000020FCF78AFDFCF71AFE3C
:10411000FCF7A4FDC820FCF78BFFFCF739FD4FF43A
:104120007A70FCF785FFFEF73BFC0F4C40F6B83089
:104130002082E081A0812083C820E08320846084E5
:10414000FDF71EFAFDF796F9FCF7FAFEFCF7A4FF5F
:10415000FDF700F8207D022803D1FEF7EBF8FDF70C
:104160003FFDFDF787FFEBE7D4010020F0B50B30F2
:10417000154D20F007010024144A0FE003688B421C
:104180000BD38B4205D95E1A43184768C3E9006711
:1041900000E04368136002C004E0021D10680028BC
:1041A000ECD12046002802D1286808B10020F0BDDB
:1041B000064A07481060074A121A22F00702C0E9AF
:1041C000002401202860D7E7640000206000002060
:1041D0009C030020980500202DE9F041074608784F
:1041E000234E5B2803D0B1600020BDE8F08105209C
:1041F000F860481C00F0DEFF044620785D2811D0EE
:10420000FFF7EEFE0546B86070B1204600F0D2FF21
:104210000146284600F084FA00F0CCFF0446200056
:1042200004D016E0601CE0E70020DEE70020DCE7B9
:10423000FFF7D6FEB0B1286045600546601C00F06F
:10424000B9FF0146284600F06BFA00F0B3FF0446C0
:1042500054B120782C28EBD020785D2806D0B460AB
:104260000020C2E70020C0E70020BEE7601CBCE7DA
:10427000540000200178A1F13002092A01D811462A
:104280000AE0A1F14102052A01D8373904E0A1F181
:104290006102052A0AD857390A01401C0178A1F1A8
:1042A0003003092B04D8303A11440EE00020704747
:1042B000A1F14103052B02D8373A114405E0A1F1E1
:1042C0006103052B0BD8573A11440A01401C0178B1
:1042D000A1F13003092B04D8303A11440EE000203C
:1042E0007047A1F14103052B02D8373A114405E08C
:1042F000A1F16103052B0AD8573A1144090140780E
:10430000A0F13002092A04D830390844704700204F
:104310007047A0F14102052A02D837390844704796
:10432000A0F16102052A02D85739084470470020DD
:10433000704700002DE9F34F85B08A4600242546DA
:1043400059490020CDE90201002637468346012065
:1043500001909AF800002D2805D154490020CDE99C
:1043600002010AF1010A9AF80000302801D10AF18D
:10437000010A9AF800003138082817D89AF8000086
:104380003038FCF778F8804689460022484B2046B2
:104390002946FBF7E2FF42464B46FBF737FF044650
:1043A0000D461AF8010F30380928E7D99AF80000AD
:1043B0002E2827D19AF80100302823D3392821D874
:1043C0000AF1010A9AF800003038FCF754F88046E8
:1043D00089460022364B20462946FBF7BEFF42465F
:1043E0004B46FBF713FF04460D4600222E4B30468A
:1043F0003946FBF7ACFF06460F461AF8010F303876
:104400000928DFD99AF80000652801D045281DD178
:104410001AF8010F2B2802D02D2803D010E00AF142
:10442000010A0DE04FF0FF3001900AF1010A07E0A8
:104430000BEB8B0100EB410B0AF1010AABF1300BE6
:104440009AF80000A0F130010929F1D901980BFB7D
:1044500000F0FCF710F832463B46FBF7D7FE024669
:104460000B460020124900F0B9F906460F46DDE977
:10447000020122462B46FBF770FF32463B46FBF714
:104480006CFF04460D460598C0E9064520462946BE
:10449000FCF702F80599486105980321C16007B04F
:1044A0005046BDE8F08F00000000F03F0000F0BF74
:1044B000000024402DE9F04107460878384E7B285B
:1044C00003D0B1600020BDE8F0810620F860481CF0
:1044D00000F070FE054628787D2818D0FFF780FD93
:1044E0000446B860A8B1284600F064FE01462046A4
:1044F00000F058F800F05EFE68B1216921620027E3
:10450000276101783A2908D0B0600020DBE7681CF9
:10451000D9E70020D7E70020D5E7401C00F04AFE8D
:104520000146204600F0FCF800F044FE0546280055
:1045300028D1C8E7FFF754FDA8B1206044600446C5
:10454000681C00F037FE0146204600F02BF800F012
:1045500031FE50B121692162276101783A2906D0E4
:10456000B0600020AFE70020ADE70020ABE7401CC3
:1045700000F020FE0146204600F0D2F800F01AFEBE
:10458000054645B128782C28D4D028787D2804D039
:10459000B560002097E7002095E7681C93E70000CE
:1045A000540000202DE9F04780460D466C1C002089
:1045B0002A785949222A06D08D60BDE8F087641C0C
:1045C0005C2A00D1641C2278222A02D00AB1401C45
:1045D000F5D10968401C88470746380004D0681C9C
:1045E0003C464FF480691AE00020E6E75C2903D0DE
:1045F00004F8011B401C12E0461C3078722825D0BC
:1046000006DC622816D0662818D06E2804D119E07E
:1046100074281FD0752821D004F8010B701C017874
:10462000222901D00029E1D100212170017822291D
:104630006AD06AE0082004F8010BEFE70C2004F8C8
:10464000010BEBE70A2004F8010BE7E70D2004F863
:10465000010BE3E7092004F8010BDFE7701CFFF70B
:1046600009FE0546361DA5F55C404845D6D3002D0C
:10467000D4D0A5F55840484513D270785C28CDD1E8
:10468000B0787528CAD1F01CFFF7F4FDB61DA0F56F
:104690005C414945C2D2C5F3090161F39F2000F591
:1046A00080350421802D01D2012108E0B5F5006F8D
:1046B00001D2022103E0B5F5803F00D2032160184A
:1046C00001291AD0022911D0032908D0042919D1AF
:1046D00005F0BF0242F0800200F8012DAD0905F09F
:1046E000BF0242F0800200F8012DAD0905F0BF02C3
:1046F00042F0800200F8012DAD09084A525C2A43BD
:1047000000F8012D441889E7401CC8F810700421F6
:10471000C8F80C1051E7000054000020B0600008F9
:1047200070B505460C46002C20D0042224A120465A
:10473000FBF75DFDE0B1052223A12046FBF757FD05
:10474000D0B1042222A12046FBF751FDC0B1207850
:1047500022281AD02D2803D0A0F1300109291AD817
:1047600021462846BDE87040FFF7E4BD002070BD3B
:104770000220E860201D70BD0020E860601D70BD53
:104780000120E8606861201D70BD21462846BDE813
:104790007040FFF707BF5B2805D07B2809D00E4883
:1047A0008460002070BD21462846BDE87040FFF7B8
:1047B00013BD21462846BDE87040FFF77BBE0000D0
:1047C0006E756C6C0000000066616C736500000023
:1047D0007472756500000000540000202DE9F04D52
:1047E0001D460C4698B0174621F0004123F00043C7
:1047F000002814BF4FF0010C4FF0000C0CEB440CE0
:10480000FE4A0CEB02064FEA620C66452BD33E00D3
:1048100018BF012606EB45061644F94A964222D3F4
:10482000F84A53EA070C02D0944205D148B918B0AF
:1048300000201146BDE8F08D002808BF4FF0000CA5
:1048400001D04FF0010C0CEB440212F5001F0AD806
:10485000002F14BF4FF0010C4FF0000C0CEB450281
:1048600012F5001F07D918B03A462B462146BDE87D
:10487000F04DFEF7F7BE0022DFF88CA3002CB8BF86
:10488000534526DADFF884C36345A8BF022220DA45
:10489000DFF870C39C451CDCDFF874C30CEB235CB1
:1048A000BCF1140F08DDCCF1340627FA06FC0CFA33
:1048B00006F6BE420DD108E05FB9CCF1140623FA2A
:1048C00006FC0CFA06F69E4203D10CF00102C2F17E
:1048D000020251EA000C19D1002D17DA002C18BF82
:1048E000022A01D0012A07D00220FEF7E3FE18B009
:1048F000BDE8F04DFEF7AEBE0220FEF7DBFEFEF790
:10490000A9FE18B081F00041BDE8F08DB7F1000CB0
:104910006CD1534525D104F1804212F5801201BFBC
:1049200000280020B74918B008BFBDE8F08DB54891
:10493000884207DC002DA1BF6046294618B0BDE8BB
:10494000F08D07E0281E05DA80F0004118B06046BF
:10495000BDE8F08DAF497944D1E9000118B0BDE858
:10496000F08DDFF8A0C2634525D1002D1FDA19B103
:10497000514512D1D8B909E0002840F0EC82A24A92
:10498000214618B062F31E01BDE8F08D00202146DB
:1049900018B060F31E01BDE8F08D08DA18B02346A8
:1049A000BDE8F04D024600206146FBF701BF18B09C
:1049B0002146BDE8F08D514518DAB5F1804F0DD094
:1049C000A5F1005CBCF1FF5C10D1B4F1000C0DDB73
:1049D00018B06146BDE8F04D00F0F6BB234618B0B4
:1049E0000246BDE8F04D1946FBF7B7BC060024F0BF
:1049F000004C3BD1D9B1514533D1002C06DD002DFF
:104A0000A1BF0020514618B0BDE8F08D002C01DD9B
:104A1000002D1BDB002C13DA002D11DB012A4FF0D7
:104A2000000014BF78497C4918B0BDE8F08D022A17
:104A300018BF002C0AD0012A08D1002C06DA0AE09F
:104A4000002CB8BF002D11DA012A04D0002018B0C4
:104A50000146BDE8F08D18B000204FF00041BDE8E0
:104A6000F08DA1F14050B0F17F601AD0012000EB31
:104A7000E47050EA020421D0624C521E4FF0000B49
:104A8000104304BF4FF0000B644C654883427CDD4B
:104A9000644A654893421FDD884217DB002D25DB01
:104AA00037E0002C00DA4AB1022A0CBF01204FF097
:104AB000FF3018B0BDE8F04DFBF7DDBC0120FEF77C
:104AC000F9FD18B0BDE8F04DFEF7CEBD4D4A8A4263
:104AD00002DC002D0ADC1CE0814202DA002D18DA2B
:104AE00004E0484B994220DD002D12DD0220FEF744
:104AF000E1FDFEF7BFFD05460E460022534658462F
:104B00002146FBF72AFC18B066F31E012846BDE8D3
:104B1000F08D0220FEF7CEFDFEF7B4FD0A462146D9
:104B200018B062F31E01BDE8F08D002230466146E8
:104B3000FBF70DFC80460E466FF00102FBF77FFC91
:104B40004FF05532394BFBF705FC42463346FBF735
:104B500004FC0022364BFBF7FDFB824642463346FF
:104B6000049110461946FBF7F8FB5246049BFBF7ED
:104B7000F4FB8A4600904FF0C0422E4B404631462F
:104B8000FBF7EBFB2C4A2B4B00E027E0CDE90601BD
:104B900051460098FBF7E1FB82460191274A284BDA
:104BA00040463146FBF7D9FB5246019BFBF7CFFB52
:104BB00082460B4602460591DDE90601FBF726FB1E
:104BC000DDE90623002688463046FBF7C0FB524647
:104BD000059BFBF7BFFB024600F07EB90020B1F554
:104BE000801F07DA352230466146FBF728FC06466F
:104BF0006FF0340000EB215024E00000FFFF1F00A5
:104C0000FFFF0F000000F03F0000F07F0000404376
:104C100001FCFFFFE61700000000F0FF0000F0BFFE
:104C20000000E0410000F043FFFFEF3F5555D53F46
:104C30000000E03F4715F73FFE822B6544DF5DF83B
:104C40000BAE543EA0F2FF300190C1F3130040F0D0
:104C50007F6141F040510291FE498842D8BF002057
:104C600004DDFD498142C8BF012001DD0D9008E04F
:104C700000200D900198401C01900298A0F5801032
:104C800002900299F54878440B910D9900EBC10010
:104C9000D0E900230F9330460A920B99FBF757FB9C
:104CA000CDE90601DDE90A2130460F9BFBF7AEFA9C
:104CB00002460B460020EA49FBF77AFD05910246C1
:104CC0000B460090DDE90601FBF747FB1490E54831
:104CD0008A464FF0000878440299006812904FF01D
:104CE000005040EA61010D980F9B01EB804000F5F8
:104CF000002109910A9A1298FBF729FB32460B9B77
:104D0000FBF728FB42465346FBF727FB064602917A
:104D100040465146099B129AFBF71FFBDDE906232B
:104D2000FBF718FB3246029BFBF711FB059B009A31
:104D3000FBF713FB0091149A049053461046194652
:104D4000FBF70BFB06460246C7480B4602910621BD
:104D50007844FEF729FCCDE90510029B3246104647
:104D60001946FBF7FAFADDE90532FBF7F6FA059189
:104D70000646534640461946149AFBF747FA009BED
:104D8000049AFBF7EAFA3246059BFBF73FFACDE9B6
:104D900005104246534610461946FBF7DEFA00223C
:104DA000B24B02910A90FBF731FADDE90532FBF7CD
:104DB0002DFA0E464246AD4B4046FBF7C8FA029B21
:104DC0000A9AFBF7C4FADDE90532FBF7C3FA42465B
:104DD00002910A90334610465146FBF7BEFACDE9E0
:104DE00006015346149A02990A98FBF7B6FA8A46C6
:104DF00002903346424600990498FBF7AEFA5346B8
:104E0000029AFBF703FA82460B4602460591DDE95A
:104E10000601FBF7FBF9DDE906230020884606467C
:104E2000FBF795FA5246059BFBF794FA82460991E7
:104E30004FF060428E4B30464146FBF78EFA0490AD
:104E400006918C4A8A4B50460999FBF786FA8246AE
:104E50000291894A894B30464146FBF77EFA524619
:104E6000029BFBF7D3F9864B7B440D9A03EBC203FD
:104E7000D3E90023FBF7CAF90E9007910198FBF7DD
:104E8000FAFA0591DDE9061382460E9A0498FBF7BB
:104E9000BDF97C4A7A440D9B02EBC303D3E900239E
:104EA00000930292FBF7B2F95246059BFBF7AEF96D
:104EB0000026884652463046059BFBF748FA009B81
:104EC000029AFBF744FA069B049AFBF740FA079B09
:104ED0000E9AFBF73FFA024600200B460290384636
:104EE0002946FBF73AFA824601912B463846194685
:104EF000029AFBF72CFA32464346FBF72EFA52464B
:104F0000019BFBF783F907468A463246434629460A
:104F10000298FBF722FA05460E463A465346FBF73F
:104F200075F9594A8846914221DBA8EB020353EAFE
:104F3000000210D12A463346FBF709FACDE90401F5
:104F4000524A534B38465146FBF760F9DDE90423DA
:104F5000FBF7EEFA21D20220FEF7ACFBFEF78AFB4C
:104F60000A46214618B062F31E01BDE8F08D494B98
:104F700028F000429A4210D3474A08EB020353EA52
:104F800000027FF4C6AD2A463346FBF7E0F93A4605
:104F90005346FBF7CDFA7FF6BCAD0022019228F014
:104FA00000403E493E4A01EB2051824223DA481C30
:104FB0004FF4801121FA00F040443A4AC0F30A51FC
:104FC0007A44394BA1F2FF31CB4020EA0303C0F30E
:104FD000130040F48010C1F11401C8401268019020
:104FE000B8F1000FBCBF4042019028463146FBF7A4
:104FF000AEF905460E462A46334638465146FBF77B
:1050000005F94FF000084246284B40460591FBF752
:10501000A4F9CDE90601264A264B40460599FBF73F
:105020009CF9009102902A46334640460599FBF7C9
:105030008EF93A465346FBF78DF91F4A1F4BFBF793
:105040008CF9009B029AFBF7E1F807468846024676
:105050000B4635E08E9803007AB60B002E14000044
:105060000000F03F661400009413000000000840A8
:1050700009C7EE3FFD033ADCF5015B14E02F3EBEAD
:105080006C1200003012000000009040FE822B6580
:105090004715973C00CC904000346F3F01FCFFFF68
:1050A0000000E03F7C110000FFFF0F00432EE63FB1
:1050B000396CA80C615C20BEEF39FAFE422EE63F47
:1050C000DDE90601FBF7A2F8DDE9062305460E46F9
:1050D000FBF73DF93A464346FBF73CF90F462A46B3
:1050E0003346009010461946FBF737F982460246D0
:1050F0002E4888460B4605217844FEF755FA52465D
:105100004346FBF72AF92A463346FBF723F9804644
:105110008A463B4628463146009AFBF71EF93B4635
:10512000009AFBF773F80691009000224FF080433D
:1051300040465146FBF70BF90F460C90424653464A
:1051400028463146FBF709F93B460C9AFBF730FB42
:10515000069B009AFBF7FBF82A463346FBF7F7F865
:105160000022134BFBF7F6F8054601980E4601EBBB
:1051700000510815002810DC28463146019AFBF73B
:105180005EF9FEF7FDF9042808BFFEF77BFA284612
:105190003146019AFBF753F905460B4618B02A46EB
:1051A00058462146BDE8F04DFBF7D7B81C1000006B
:1051B0000000F03F00E0401C002804D001780029E6
:1051C00001D02029F7D970472DE9F04106460F4656
:1051D000FBF788FB041E0D4618BF0120284320F072
:1051E0000040C0F17F6000F1E040C00F0ED0301CE5
:1051F00018BF0120384320F00040C0F17F6000F16B
:10520000E040C00F04BF0120FEF754FA20462946B3
:10521000BDE8F08100000000000000000000000078
:10522000000000003F4000000000000000003000CF
:10523000400030004000000009000BC03D000BC0E2
:105240003D00090018C024407FE02240318000006A
:10525000180024C01B000D803240018003801C40D8
:1052600027401C8007400040100060000000000044
:10527000000000000000000000001F8020404020CF
:105280000000402020401F800000000009000600B0
:105290001F80060009000000040004003F80040095
:1052A000040000000010006000000000000000008A
:1052B000040004000400040004000000000000409A
:1052C0000000000000000000002001C006003800BF
:1052D000400000001F802040204020401F80000030
:1052E000000010403FC000400000000018C02140F6
:1052F00022402440184000001080204024402440D8
:105300001B80000002000D0011003FC001400000A2
:105310003C80244024402440238000001F802440FF
:1053200024403440038000003000200027C03800B3
:10533000200000001B802440244024401B800000EB
:105340001C0022C0224022401F80000000000000FC
:1053500008400000000000000000000004600000A1
:1053600000000000000004000A00110020804040FE
:105370000900090009000900090000000000404080
:10538000208011000A00040018002000234024009F
:10539000180000001F802040274029401F400000C7
:1053A000004007C039000F0001C0004020403FC04E
:1053B000244024401B8000001F80204020402040CB
:1053C0003080000020403FC0204020401F8000006F
:1053D00020403FC024402E4030C0000020403FC04D
:1053E00024402E00300000000F001080204022409A
:1053F0003380020020403FC0040004003FC0204032
:10540000204020403FC0204020400000006020207D
:1054100020203FC02000200020403FC024400B003F
:1054200030C0204020403FC020400040004000C02D
:105430003FC03C0003C03C003FC0000020403FC0D4
:105440000C4023003FC020001F802040204020400F
:105450001F80000020403FC02440240018000000AE
:105460001F802140214020E01FA0000020403FC0BD
:105470002440260019C0004018C024402440224087
:1054800031800000300020403FC02040300000004C
:1054900020003F80004000403F80200020003E0070
:1054A00001C0070038002000380007C03C0007C0DA
:1054B00038000000204039C0060039C020400000FC
:1054C0002000384007C0384020000000304021C094
:1054D0002640384020C00000000000007FE040204F
:1054E00040200000000070000C000380004000001D
:1054F0000000402040207FE000000000000020006D
:1055000040002000000000000010001000100010FB
:10551000001000100000000040000000000000002B
:10552000000002800540054003C0004020003FC04D
:105530000440044003800000000003800440044055
:105540000640000000000380044024403FC00040AB
:1055500000000380054005400340000000000440B7
:105560001FC0244024402000000002E005500550E8
:105570000650042020403FC00440040003C0004007
:105580000000044027C00040000000000010001090
:10559000041027E00000000020403FC00140070049
:1055A00004C00440204020403FC0004000400000B4
:1055B00007C0040007C0040003C00000044007C087
:1055C0000440040003C00040000003800440044085
:1055D00003800000041007F0045004400380000022
:1055E000000003800440045007F00010044007C08E
:1055F0000240040004000000000006400540054091
:1056000004C00000000004001F80044000400000AF
:10561000040007800040044007C000400400070069
:1056200004C0018006000400060001C0070001C09C
:1056300006000000044006C0010006C0044000004F
:105640000410071004E0018006000400000004407C
:1056500005C00640044000000000000004007BE09C
:1056600040200000000000000000FFF000000000EB
:10567000000040207BE004000000000040008000AB
:10568000400020002000400000000000000000005A
:1056900000000000000000000000000000001FCC1F
:1056A000000C000000000000000008003000600056
:1056B0000800300060000000022003FC1E200220D1
:1056C00003FC1E200220000000000E1811043FFF02
:1056D00010840C78000000000F0010840F3800C008
:1056E000077818840078000000780F8410C4112413
:1056F0000E9800E4008400080800680070000000B4
:10570000000000000000000000000000000007E0B2
:10571000181820044002000000004002200418185D
:1057200007E00000000000000240024001800FF08E
:1057300001800240024000000080008000800FF8DD
:1057400000800080008000000001000D000E0000BD
:1057500000000000000000000000008000800080C9
:1057600000800080008000800000000C000C000021
:1057700000000000000000000000000600180060AB
:105780000180060018002000000007F0080810043F
:105790001004080807F000000000080408041FFCBB
:1057A000000400040000000000000E0C101410247F
:1057B000104411840E0C000000000C181004110499
:1057C000110412880C700000000000E00320042483
:1057D00008241FFC0024000000001F9810841104FE
:1057E0001104108810700000000007F008881104F0
:1057F000110418880070000000001C00100010FC4C
:1058000013001C001000000000000E38114410842A
:10581000108411440E38000000000700088C10446A
:105820001044088807F00000000000000000030C8E
:10583000030C000000000000000000000001010651
:105840000000000000000000000000800140022075
:105850000410080810040000022002200220022088
:10586000022002200220000000001004080804109A
:10587000022001400080000000000E001200100C09
:10588000106C10800F00000003E00C1813E41424C7
:1058900017C4082807D000000004003C03C41C40C3
:1058A000074000E4001C000410041FFC1104110454
:1058B00011040E880070000003E00C18100410049E
:1058C000100410081C10000010041FFC1004100429
:1058D0001004080807F0000010041FFC1104110454
:1058E00017C410040818000010041FFC1104110054
:1058F00017C010000800000003E00C18100410048A
:1059000010441C780040000010041FFC108400802C
:10591000008010841FFC10040000100410041FFC01
:105920001004100400000000000300011001100129
:105930001FFE10001000000010041FFC1104038063
:105940001464181C1004000010041FFC1004000450
:1059500000040004000C000010041FFC1F0000FCE9
:105960001F001FFC1004000010041FFC0C040300A7
:1059700000E010181FFC100007F0080810041004C5
:105980001004080807F0000010041FFC10841080A9
:10599000108010800F00000007F008181024102459
:1059A000101C080A07F2000010041FFC110411006B
:1059B00011C011300E0C000400000E1C11041084E4
:1059C000108410441C3800001800100010041FFC44
:1059D000100410001800000010001FF8100400044C
:1059E000000410041FF8100010001E0011E0001C3D
:1059F000007013801C0010001FC0103C00E01F004E
:105A000000E0103C1FC000001004180C163401C048
:105A100001C01634180C100410001C00130400FC04
:105A200013041C00100000000804101C10641084F3
:105A300013041C04101800000000000000007FFE8A
:105A40004002400240020000000030000C000380D1
:105A50000060001C00030000000040024002400201
:105A60007FFE000000000000000000002000400059
:105A70004000400020000000000100010001000182
:105A80000001000100010001000040004000200072
:105A90000000000000000000000000980124014404
:105AA0000144014400FC000410001FFC00880104B4
:105AB00001040088007000000000007000880104EC
:105AC0000104010400880000000000700088010447
:105AD000010411081FFC0004000000F80144014407
:105AE0000144014400C800000000010401040FFC4F
:105AF0001104110411001800000000D60129012929
:105B0000012901C90106000010041FFC00840100E6
:105B10000100010400FC000400000104190419FC48
:105B20000004000400000000000000030001010167
:105B3000190119FE0000000010041FFC00240040A1
:105B400001B4010C010400000000100410041FFC4B
:105B50000004000400000000010401FC0104010035
:105B600001FC0104010000FC010401FC00840100AF
:105B70000100010400FC0004000000F8010401041D
:105B80000104010400F80000010101FF0085010487
:105B9000010400880070000000000070008801040B
:105BA0000104010501FF00010104010401FC00845E
:105BB0000104010001800000000000CC0124012448
:105BC000012401240198000000000100010007F8F1
:105BD0000104010400000000010001F800040004B9
:105BE0000004010801FC0004010001800170000CA8
:105BF000001001600180010001F0010C003001C0C3
:105C00000030010C01F0010000000104018C00745F
:105C10000170018C01040000010101810171000E7D
:105C2000001801600180010000000184010C0134B2
:105C300001440184010C000000000000000000008D
:105C400001003EFC40024002000000000000000095
:105C5000FFFF0000000000000000400240023EFC88
:105C600001000000000000000000600080008000D3
:105C700040004000200020000000000FFFF80FFF50
:105C8000F80C0C000C0C000C0C00040C00060C00B2
:105C9000061C0003F80001F0000000000000000FE7
:105CA000FFF80FFFF80FF00000FF800007F8000773
:105CB000F801FF000FE0000FFFF80FFFF8000000F1
:105CC0000000000180100780700600F00C01D00C6D
:105CD00003900C07100E1C1007F81003E0100000D2
:105CE0001000000000000000000000003800003834
:105CF00000000000000000000000000000000000A4
:105D000000000000000000000000800038E007F8FC
:105D10007007B01004201804201804301804303024
:105D2000043CF0041FE0000300000000000000003D
:105D3000000003FC0000003FFFC000007FFFF000F8
:105D400000FC01F80001E000780003C0001C000323
:105D500080001C000300000E000300000E00038002
:105D6000001C0003C0003C0001F000780000FFFFB1
:105D7000F000007FFFE000000FFF000000000000C7
:105D80000000000000000000000000000000000013
:105D90000000000000001C000000001800000000CF
:105DA00038000000007000000000E000000001FF6B
:105DB000FFFC0003FFFFFC0003FFFFFC00000000EE
:105DC00000000000000000000000000000000000D3
:105DD00000000000000000000000000000000000C3
:105DE000000000000000100000000070001C000017
:105DF000F8003C0001E0007C0003C000FC000380D0
:105E000001EC00038003CC0003800F0C0003801E14
:105E10000C0003803C0C000380F80C0001E7E00C50
:105E20000001FFC00C0000FF000C000018000C0077
:105E30000000000000000000000000000000000062
:105E400000008000003000E000007000F00001F071
:105E500000780001C0003C000380001C000380604B
:105E60000C000300E00C000300E00C000380E01CC9
:105E7000000381F01C0001E7B8780001FF3FF80043
:105E800000FE1FF000001807C00000000000000026
:105E900000000000000003800000000780000000F8
:105EA0001F800000003F800000007B80000001E3B5
:105EB00080000003C38000000F838000001E038069
:105EC00000007C03800000F003800003FFFFFC0063
:105ED00003FFFFFC0003FFFFFC0000000380000045
:105EE00000038000000003800000000000000000AC
:105EF000000000000020E0000007E0F00000FFE0EC
:105F0000780003FFC01C0003F1801C000383800E97
:105F1000000383800E000383800E000383800C0047
:105F20000383801C000381C03C000381E0780003F0
:105F300080FFF80003807FE00000001F8000000069
:105F4000000000000000000000000000000000074A
:105F5000000000003FE0000000FFF0000003F8F840
:105F6000000007E03C00001FC01C00003F800C0048
:105F700000F9800E0001F1800E0003C1800E0003C5
:105F800001C00C000201C01C000000E07C00000009
:105F9000FFF80000007FF00000001FC000000000BC
:105FA000000000000000000000000000038000006E
:105FB00000038000000003800000000380001C003C
:105FC000038000FC00038007FC0003801FE0000347
:105FD000807F00000381F800000387E00000039F3A
:105FE00000000003FC00000003F000000003E000DC
:105FF000000003800000000000000000000000001E
:1060000000000007E000007E1FF00000FFBFF80066
:1060100001E7F83C000381F01C000380E00C000362
:1060200080E00E000300E00E000380E00E0003801D
:10603000E00C000381F01C0001E7B83C0000FF3FCA
:10604000F800007E1FF00000000FE00000000000DC
:106050000000000000000000000000003FC0000041
:10606000007FE0000000FFF0000001E07800000386
:10607000C03806000380181E000380187E000380CD
:1060800019F80003801FE00003803FC00003C07FB9
:10609000000001E1FC000000FFF00000007FC000F4
:1060A00000003F00000000000000000000000000B1
:1060B0000000C0E0F0F8FC00000000000000F03F2D
:1060C000000000000000F83F000000000000000099
:1060D0000000004003B8E23F0000000000000000A4
:1060E00006D0CF43EBFD4C3E033333333333E33F32
:1060F000FFAB6FDBB66DDB3F4D268F515555D53F5E
:1061000001411DA96074D13F65DBC9934A86CD3F2B
:10611000EF4E454A287ECA3F3E5555555555C53F19
:1061200093BDBE166CC166BF2CDE25AF6A56113F0B
:10613000F16BD2C541BDBBBED0A4BE726937663E0D
:10614000000000000000000068610008000000205E
:106150006C00000094360008D46100086C00002038
:106160002C090000A436000800A24A040000000028
:1061700000000000010203040607080902040608E3
:1061800000000000010203040102030406070809DD
:1061900000000000000000000000000000000000FF
:1061A00000000000010000000000000000000000EE
:1061B0000000000000000000FFFF00006D4100082B
:1061C000B9400008000000000000000000000000CE
:0461D00000000000CB
:0400000508000131BD
:00000001FF
